:1000000004EF00F0FFFFFFFFC8EC03F04E0E00010D
:10001000816F6F0E826F6B0E836F690E846F610E3E
:10002000856F5F0E866F4C0E876F430E886F440E90
:10003000896F5F0E8A6F310E8B6F380E8C6F460E94
:100040008D6F320E8E6F350E8F6F320E906F916BFB
:10005000560E926F650E936F720E946F730E956FBE
:10006000750E966F730E976F200E986F300E996F06
:10007000330E9A6F200E9B6F6D0E9C6F610E9D6FFD
:10008000690E9E6F200E9F6F310EA06F300EA16F14
:10009000A26B410EA36F440EA46F430EA56F200EFA
:1000A000A66F430EA76F480EA86F300EA96F3D0EC6
:1000B000AA6FAB6B410EAC6F440EAD6F430EAE6FCB
:1000C000200EAF6F430EB06F480EB16F310EB26F9E
:1000D0003D0EB36FB46B560EB56F610EB66F6C0EFE
:1000E000B76F750EB86F650EB96F200EBA6F3D0E03
:1000F000BB6FBC6B500EBD6F610EBE6F750EBF6FD8
:100100006C0EC06F660EC16F6A0EC26F750EC36F44
:100110006A0EC46F6F0EC56F400EC66F660EC76F56
:10012000720EC86F650EC96F650ECA6F660ECB6F13
:10013000720ECC6FCD6B816A120E936EF19EFF0E24
:10014000806EFF0E926E010EC26E810EC16E946AB9
:100150000A0EAF6EAC8495EC05F0819E08EC02F0BF
:10016000020E0C6EFF0E0B6EFF0E0A6E0C2E01D0EF
:1001700007D00B2E01D003D00A2EFED7FAD7F6D720
:10018000460E0B6EFF0E0A6E0B2E01D003D00A2E08
:10019000FED7FAD7CF0E0A6E0A2EFED70000406AAD
:1001A000416A84EC05F015C035F016C036F0810EBA
:1001B000376E000E386EDAEC04F000C015F001C0A6
:1001C00016F003EC04F0176A0001CE6B79EC02F034
:1001D000406A010E416E84EC05F015C035F016C082
:1001E00036F0920E376E000E386EDAEC04F000C076
:1001F00015F001C016F003EC04F015C035F016C080
:1002000036F0A30E376E000E386EDAEC04F000C044
:1002100015F001C016F0406A020E416E84EC05F044
:10022000356A66EC04F000C033F001C034F000C061
:1002300035F001C036F031C037F032C038F0E7ECAD
:1002400002F015C035F016C036F031C037F032C0BC
:1002500038F036EC04F003EC04F0010E176E03ECFA
:1002600004F0176A15C035F016C036F0AC0E376EC4
:10027000000E386EDAEC04F000C015F001C016F084
:10028000406A030E416E84EC05F0010E356E66EC9B
:1002900004F000C033F001C034F000C035F001C0FC
:1002A00036F031C037F032C038F0E7EC02F015C05C
:1002B00035F016C036F031C037F032C038F036ECC9
:1002C00004F003EC04F0010E176E03EC04F0176A5F
:1002D0000001CE51010F046E04C0CEF00450000A9C
:1002E00004E179EC02F00001CE6BFF0ECE15006E3A
:1002F000000ECEBFFF0E016E000E011600C033F0DF
:1003000001C034F000C035F001C036F015C037F040
:1003100016C038F0E7EC02F0406A040E416E84EC3F
:1003200005F003EC04F0406A050E416E84EC05F024
:1003300015C035F016C036F0B50E376E000E386EAB
:10034000DAEC04F000C015F001C016F053EC05F033
:1003500000C033F001C034F000C035F001C036F009
:1003600031C037F032C038F0E7EC02F015C035F09C
:1003700016C036F031C037F032C038F036EC04F039
:1003800003EC04F0010E176E03EC04F0176A406AE8
:10039000070E416E84EC05F015C035F016C036F03E
:1003A000BD0E376E000E386EDAEC04F000C015F0AA
:1003B00001C016F003EC04F0046A81BE042A045064
:1003C000000A03E1818EE6EF01F0819E040E0C6EBF
:1003D000FF0E0B6EFF0E0A6E0C2E01D007D00B2EF7
:1003E00001D003D00A2EFED7FAD7F6D7300E0B6E07
:1003F000FF0E0A6E0B2E01D003D00A2EFED7FAD7BD
:10040000880E0A6E0A2EFED700000000E1D6FFD744
:10041000828482808294030E0C6EFF0E0B6EFF0EA0
:100420000A6E0C2E01D007D00B2E01D003D00A2E5D
:10043000FED7FAD7F6D78C0E0B6EFF0E0A6E0B2E78
:1004400001D003D00A2EFED7FAD7A10E0A6E0A2ECB
:10045000FED700008284210E426E6CEC05F0900EF7
:10046000426E6CEC05F0050E426E6CEC05F0130E5E
:10047000426E6CEC05F0200E426E6CEC05F0210E25
:100480000B6EFF0E0A6E0B2E01D003D00A2EFED784
:10049000FAD7600E0A6E0A2EFED7000000000C0E7E
:1004A000426E6CEC05F0B4EC04F0020E0C6EFF0E24
:1004B0000B6EFF0E0A6E0C2E01D007D00B2E01D052
:1004C00003D00A2EFED7FAD7F6D7460E0B6EFF0ED4
:1004D0000A6E0B2E01D003D00A2EFED7FAD7CF0E0C
:1004E0000A6E0A2EFED70000406A416A84EC05F0CD
:1004F00012008196818A818481868180818A010EA1
:10050000356E000E366E800E006E800E3618005C62
:1005100002E1355005080BE3100E3B6E8EEC04F043
:10052000FF0E3B6E8EEC04F0354A362AECD7100EE7
:100530003B6E8EEC04F03B6A8EEC04F0040E0C6E05
:10054000FF0E0B6EFF0E0A6E0C2E01D007D00B2E85
:1005500001D003D00A2EFED7FAD7F6D7300E0B6E95
:10056000FF0E0A6E0B2E01D003D00A2EFED7FAD74B
:10057000880E0A6E0A2EFED700000000100E3B6E99
:100580008EEC04F0440E3B6E8EEC04F0040E0C6E08
:10059000FF0E0B6EFF0E0A6E0C2E01D007D00B2E35
:1005A00001D003D00A2EFED7FAD7F6D7300E0B6E45
:1005B000FF0E0A6E0B2E01D003D00A2EFED7FAD7FB
:1005C000880E0A6E0A2EFED700000000120037C007
:1005D000E1FF38C0E2FF200EE66E010E3724E16E27
:1005E000000E3820E26E200EE66E020E3724E16E19
:1005F000000E3820E26E200EE66E030E3724E16E08
:10060000000E3820E26E200EE66E040E3724E16EF6
:10061000000E3820E26E300EE66E050E3724E16ED5
:10062000000E3820E26EE66A040E396E000E006E8F
:100630003650005C02E13550000828E2395037247A
:10064000E16E000E3820E26E0A0E046E000E056E9A
:1006500035C000F036C001F0FFEC04F008C000F037
:1006600009C001F0300E002600C0E6FF0A0E046E3D
:10067000000E056E35C000F036C001F0FFEC04F04E
:1006800000C035F001C036F03906D0D71200200E78
:100690003B5C03E33B507F08D8A01200050E3B02F1
:1006A000F3CF3CF0F4CF3DF0A00E3C5E000E3D5A7F
:1006B000050E3E6E000E3F6E800E006E800E3F18DF
:1006C000005C02E13E5000081FE2700E3C24006E08
:1006D0000B0E3D20016E000E026E000E3DBEFF0EA1
:1006E0000222000E00C0F6FF01C0F7FF02C0F8FFB3
:1006F0000900F5CF40F0ABEC05F03C4A3D2A010E75
:100700003E5E000E3F5AD8D7406AABEC05F01200AF
:1007100081943C6A3D6A3E6A3F6A0F0E3B6E800ED2
:100720003B18006E800E000A005C28E3819A818AE3
:10073000046A81B8042A0450010A1EE13B04006ED9
:10074000000E3BBEFF0E016E000E015A00C004F009
:10075000010E006E000E016E045005E000360090A0
:100760000136FF0FFAD700503C2601503D22000E03
:1007700001BEFF0E3E223F223B06D1D781843CC002
:1007800000F03DC001F03EC002F03FC003F0120097
:10079000310E186E320E196E330E1A6E340E1B6E39
:1007A000350E1C6E360E1D6E370E1E6E380E1F6E09
:1007B000390E206E300E216E310E226E320E236EF7
:1007C000330E246E340E256E350E266E360E276ED1
:1007D0002E0E286E296A180E156E000E166E310E3A
:1007E0002A6E320E2B6E330E2C6E340E2D6E350E9D
:1007F0002E6E360E2F6E306A2A0E316E000E326E5D
:10080000000E176E120015C03BF016C03CF03AEC1B
:1008100005F000C036F0356A35501524E96E000E3B
:1008200035BEFF0E1620EA6EEECF37F01750010AE4
:1008300005E137C03BF0A0EC05F004D037C03BF039
:1008400047EC03F0352A800E3518006E800E3618FE
:10085000005CE2E31750010A08E10A0E3B6EA0ECCF
:1008600005F00D0E3B6EA0EC05F0120035C039F01E
:1008700036C03AF039C0E9FF3AC0EAFFEECF00F0E7
:10088000005203E0394A3A2AF5D739C002F03AC09B
:1008900003F0394A3A2A37C0E9FF38C0EAFF374A3D
:1008A000382AEECF00F002C0E1FF03C0E2FF00C033
:1008B000E6FF02C0E9FF03C0EAFFEECF00F00052FE
:1008C000E4E135C000F036C001F01200C26AC00E8B
:1008D000C212C18CC18E35C000F0003600900036C7
:1008E0000090003600900050C212C280B3EC05F0B8
:1008F000C284C2B4FED7080E026EC4CF00F0000E50
:10090000016E025005E0003600900136FF0FFAD765
:10091000C3500012000E0112C29012008194010E09
:100920003C6E800E080A006E800E3C18005C19E3D5
:10093000819A800E3B14016E000E3BBEFF0E026ECC
:10094000000E0216000E021802E1800E011803E1EB
:100950008180ACEF04F081903B363B90818A3C2A49
:10096000E0D78184818A1200406A416A84EC05F0F4
:100970003B6A3C6A800E030A006E800E3C18005CE5
:1009800002E13B50800815E3406AABEC05F0040E31
:100990000B6EFF0E0A6E0B2E01D003D00A2EFED76F
:1009A000FAD73B0E0A6E0A2EFED700003B4A3C2ABD
:1009B000E1D7120035C039F036C03AF039C002F044
:1009C0003AC003F0394A3A2A37C0E9FF38C0EAFF93
:1009D000374A382AEECF00F002C0E1FF03C0E2FF41
:1009E00000C0E6FF02C0E9FF03C0EAFFEECF00F05F
:1009F0000052E4E135C000F036C001F01200000101
:100A0000086A096A100E0C6E013408360936045063
:100A1000085E0550D8A0053C095ED8B017EF05F078
:100A2000045008260550D8B0053C0926D890003659
:100A300001360C2E04EF05F01200446A456A800E60
:100A40004518006E800E005C02E1080E445C11E265
:100A50008296800E4314016E0150800A03E1828861
:100A600033EF05F08298828643364390444A452A04
:100A7000E6D712003BC03DF03CC03EF03DC0E9FF70
:100A80003EC0EAFF3D4A3E2AEECF00F00052F6E1BA
:100A90003B503D5C006E3C503E58016E010E005EC6
:100AA000000E015A1200046A81B2042A0450010A9D
:100AB000FAE0046A81B2042A0450000AFAE0046AE7
:100AC00081B2042A0450010AFAE0380E3B6E8EEC23
:100AD00004F088EC03F012008292829042C043F04E
:100AE0001DEC05F0210E0B6EFF0E0A6E0B2E01D0D1
:100AF00003D00A2EFED7FAD7600E0A6E0A2EFED752
:100B00000000000082801200070E4114006E400EAB
:100B10000010426E6CEC05F07F0E4014006E800EEB
:100B20000010426E6CEC05F01200AC8A900EAB6EB9
:100B3000948E949C9EAA03D0AECF39F0FBD71200BE
:100B4000016AACB2012A0150000A02E10000F8D7A4
:100B50003BC0ADFF12008282829040C043F01DEC8A
:100B600005F082801200120E0A6E0A2EFED71200C5
:100B7000000000000000005F0000000700070014F4
:100B80007F147F14242A7F2A1223130864623649B3
:100B90005522500005030000001C224100004122A4
:100BA0001C0014083E081408083E080800503000D5
:100BB000000808080808006060000020100804020F
:100BC0003E5149453E00427F400042615149462125
:100BD00041454B311814127F1027454545393C4A91
:100BE00049493001710905033649494936064949E1
:100BF000291E003636000000563600000814224137
:100C0000001414141414004122140802015109069E
:100C1000324979413E7E1111117E7F494949363E64
:100C2000414141227F4141221C7F494949417F097D
:100C30000909013E4149497A7F0808087F00417F40
:100C400041002040413F017F081422417F40404045
:100C5000407F020C027F7F0408107F3E4141413EED
:100C60007F090909063E4151215E7F09192946463F
:100C70004949493101017F01013F4040403F1F2068
:100C800040201F3F4038403F63140814630708703A
:100C900008076151494543007F41410002040810A3
:100CA000200041417F0004020102044040404040D6
:100CB000000102040020545454787F4844443838DA
:100CC00044444420384444487F3854545418087EDF
:100CD0000901020C5252523E7F0804047800447D00
:100CE00040002040443D007F1028440000417F40E8
:100CF000007C041804787C080404783844444438A0
:100D00007C14141408081414187C7C080404084883
:100D100054545420043F4440203C4040207C1C203C
:100D200040201C3C4030403C44281028440C50508B
:100D3000503C4464544C44000836410000007F009D
:100D4000000041360800100808100878464146782F
:020000040030CA
:0E000000FFF9FEFEFFFFFBFFFFFFFFFFFFFF0C
:00000001FF
